:10000000830100308A0004280C3084000D30192050
:100010000D308400263019200330B200FC30B100CE
:10002000263084002A301D2083016E2904068001B9
:10003000840A0406031D16280034AA002720800025
:10004000840A04082A06031D1E280034B100B21BCE
:10005000302832088A003108B10A0319B20A820036
:100060008313321883173108B10A8400000808008E
:100070008207FF348F348A348634833480347D346D
:100080007A3478347634733471346F346D346B343D
:100090006934683466346434623461345F345D34A6
:1000A0005C345A3458345734553454345234503400
:1000B0004F344D344C344A34483447344534443456
:1000C000423440343F343D343B343A3438343634AF
:1000D0003434333431342F342D342B342934263412
:1000E000243422341F341C341934163412340D34A1
:1000F0000834820701343F340234013401340034BF
:100100000234013401343F34023401340134003408
:100110000234013401343F340234013401340034F8
:100120000234033401343F340234033401340034E4
:100130000234033401343F340234033401340034D4
:100140000234033401343F340234033401340034C4
:1001500002340334003482072834633429342034D1
:1001600045347534673465346E3465342034533423
:100170006F346C346F347334683465346E346B347C
:100180006F3420343C3473346F346C346F347334D4
:100190006834403475346B3472342E346E346534C4
:1001A00074343E34003482070234013403340234A0
:1001B0000234013400340034820703340234023440
:1001C0000134003402340134003482070134013434
:1001D0007A340034DD3400348207F4340034FA34E5
:1001E0000034D43400348207033402340834043435
:0A01F00000348207033404340034A5
:080200008207033404340034CA
:100262000C1A4129160A031D38298312402916083F
:1002720083120102031C080086150000000086118B
:100282000314831208000C1A5429150A031D4B2962
:1002920083125329150883120102031C0800061554
:1002A2000000000006110314831208001408AC00B9
:1002B200AD010310AC0DAD0D0310AC0DAD0DFF3053
:1002C200AC07031CAD07AA013F30AB00B0232E08D8
:1002D200A1002F08A2008312080064008312860185
:1002E2008501053083168100043085007030860058
:1002F2000C12FF3096009500303094008312572183
:100302000B3098009701930192018C1005198C14FF
:1003120064000C108C180C148C10831205198C14A8
:100322000C1C9529013096290030AA008C1C9B29AF
:1003320001309C290030AA06031989298312810100
:10034200BB210C118C11B3290C19AC298312442145
:100352000C1103180C158C19B329831231218C113D
:1003620003188C150C1DA5298C1DA5298312E622C4
:10037200212286292808A300A908031DCB2983125C
:1003820006087039A800230603190800A901A90A62
:100392008D010800290B1F2A831206087039A80054
:1003A2002306031D1E2A8D0A0D08033A031D0800A9
:1003B2002808703A03191E2A2808603A031DF429F6
:1003C200103014020318E729940A182A1408AA0004
:1003D2000310AA0C03102A0C940771301402031C98
:1003E200182A70300A2A2808503A031D0C2A1130A4
:0E03F2001402031C042A1408AA000310AA0C0B
:1004000003102A0C9402182A94031408033A031DBB
:10041000182A04309400182A2808303A031D182A94
:100420000C120B309800970A1708033A031997012A
:1004300093019201A701A60183125721A9018312FA
:10044000080000308A0017081707AA00EC20A40053
:100450002A0AEC20A500270B342A910B342A140811
:100460009100900B342AA7012708023A031D552A50
:10047000FF309F07031CA00320081F04031D422A0E
:10048000A701552A21089D0703189E0A22089E07E6
:1004900000308A001E08AB001D08AA008030AA07A1
:1004A0000318AB0A2B08382096002708033A031DCF
:1004B000762AFF309F07031CA00320081F04031D9A
:1004C000632AA701762A21089D02031C9E032208A5
:1004D0009E0200308A001E08AB001D08AA00803072
:1004E000AA070318AB0A2B0838209600A708031D9B
:1004F000E42A130824078312B1002508B20031084A
:100500000318B20A2620A300930AA308031D8A2A0F
:100510009301792A230B9D2A13082407B10025088B
:10052000B20031080318B20A2620AA0000308A005F
:100530002A0838209600930A792A2308023A031DD4
:10054000B12A13082407B1002508B20031080318A6
:10055000B20A26209000930A14089100A701A70A66
:10056000E42A2308033A031DC82A9D019E0139206D
:1005700096001408AA00AB010310AA0DAB0D0310DE
:10058000AA0DAB0D2A089F002B08A0000230E32A19
:100590002308043A031DE42A00309D003F309E00EA
:1005A00000308A003F30382096001408AA00AB01C2
:1005B0000310AA0DAB0D0310AA0DAB0D2A089F0066
:1005C0002B08A0000330A7008312080000308A0027
:1005D00017081707AA00E520A4002A0AE520A500AD
:1005E000260BF92A8F0BF92A14088F008E0BF92A93
:1005F000A6012608023A031D1A2BFF309B07031C95
:100600009C031C081B04031D072BA6011A2B2108A1
:10061000990703189A0A22089A0700308A001A08D4
:10062000AB001908AA008030AA070318AB0A2B08F0
:10063000382095002608033A031D3B2BFF309B070B
:10064000031C9C031C081B04031D282BA6013B2B29
:1006500021089902031C9A0322089A0200308A009A
:100660001A08AB001908AA008030AA070318AB0AC1
:100670002B0838209500A608031DAE2B120824076E
:100680008312B1002508B20031080318B20A2620EF
:10069000A300920AA308031D542B980A18081A3ABB
:1006A00003190C1692013E2B230B672B120824070B
:1006B000B1002508B20031080318B20A2620AA00AA
:1006C00000308A002A0838209500920A3E2B230821
:1006D000023A031D7B2B12082407B1002508B20043
:1006E00031080318B20A26208E00920A14088F00DF
:1006F000A601A60AAE2B2308033A031D922B9901EB
:100700009A01392095001408AA00AB010310AA0D24
:10071000AB0D0310AA0DAB0D2A089B002B089C0003
:100720000230AD2B2308043A031DAE2B0030990094
:100730003F309A0000308A003F303820950014087E
:10074000AA00AB010310AA0DAB0D0310AA0DAB0D4F
:100750002A089B002B089C000330A6008312080087
:10076000B001AB1FBA2BAA09AA0A0319AB03AB0944
:100770003017B0172D088039B006AD1FC62BAC0955
:10078000AC0A0319AD03AD09C62BB001AE01AF0130
:100790002C082D04031900341F30B0040310B00AD4
:1007A000AC0DAD0D031CCF2BAD0CAC0C2D082B02EA
:1007B000031DDC2B2C082A02031CE42B2C08AA02A4
:1007C0002D08031C2D0AAB02AE0DAF0DB00BB01AF5
:1007D000D42BB01FF02BAE09AE0A0319AF03AF093B
:1007E0002E08AC002F08AD00301F0034AA09AA0A59
:1007F0000319AB03AB090034003400347034003407
:084000000000000000000200B6
:02400E00F53F7C
:00000001FF
